:020000040000FA
:060000002FEF09F01200D1
:060800002FEF09F01200C9
:06082A0001009212000023
:0808300000010000D0000000EF
:08083800D9CFE6FFE1CFD9FFA3
:10084000040EE126DE6ADE6ADE6ADD6ADD52DD5212
:10085000FD0EDBCF00F0FE0EDBCF01F0026A036A73
:1008600001AE02D002680368D9CFE9FFDACFEAFF10
:10087000030EEB500318E8AE02D0033408D000504A
:10088000EE5C0150EE580250EE580350EE580FE265
:100890000C0EE66E0FEC09F0E552D9CFE9FFDACF86
:1008A000EAFFEE2A000EEE22EE22EE22D1D7040E4F
:1008B000E15C02E2E16AE552E16EE552E7CFD9FF81
:1008C00012000F0EC16E070EB46E936A300E926E58
:1008D0000F0E946EF19E1200D9CFE6FFE1CFD9FF43
:1008E000020EE1268250020B01E0010E080DF3CF4B
:1008F00002F08250010B040DF3CF01F08050200B69
:1009000001E0010EE824006E8050100B01E0010EA2
:10091000002401240224DE6EDD6ADECF00F0DDCF8C
:1009200001F000C0F3FF01C0F4FF020EE15C03E23E
:1009300000D0E16AE552E16EE552E7CFD9FF12003F
:100940008092320EE66E3DEC09F0E5528084320E64
:10095000E66E3DEC09F0E5528094320EE66E3DEC19
:1009600009F0E55212008082010EE66EE66A64DF4D
:10097000E552E5528084010EE66EE66A5DDFE552DF
:10098000E5528094010EE66EE66A56DFE552E552C6
:100990001200380E816ED4DF320EE66EE66A4CDF4E
:1009A000E552E552010E816ECBDF320EE66EE66A4D
:1009B00043DFE552E5520D0E816EC2DF320EE66E68
:1009C000E66A3ADFE552E552060E816EB9DF320E75
:1009D000E66EE66A31DFE552E5521200010E816EE5
:1009E000AFDF0A0EE66EE66A27DFE552E552120037
:1009F000D9CFE6FFE1CFD9FF020E816EA1DF0A0E4B
:100A0000E66EE66A19DFE552E552FD0EDBCFE6FF42
:100A1000FE0EDB50280DF350E552E724E76EFE0E84
:100A2000E7CFDBFFFD0EDB6AFE0EDB50F36EFD0E43
:100A3000DBCFF4FFF350F45C0BE2140E816E80DF29
:100A4000320EE66E3DEC09F0E552FD0EDB2AECD7E6
:100A5000E552E7CFD9FF1200D9CFE6FFE1CFD9FFAA
:100A6000FE0EDB50816E7FDF010EE66EE66AE4DE8D
:100A7000E552E552E552E7CFD9FF1200D9CFE6FFA4
:100A8000E1CFD9FFFD0EDBCFE9FFFE0EDBCFEAFFA2
:100A9000EF500EE0FD0EDBCFE9FFDB2AFE0EDBCFD1
:100AA000EAFF01E3DB2AEF50E66ED6DFE552EAD734
:100AB000E552E7CFD9FF12000101D46B300E926EE0
:100AC000F00E936EEF0ED06FD0C181FF040ED16F88
:100AD000D151000821E2D051FE0BE842D06FD0C1C5
:100AE00081FF050EE66EE66AA7DEE552E55281500B
:100AF000100B09E08150200B06E08150400B03E011
:100B00008150800B01E10AD80101D40502E1D551E1
:100B100004D0D105D16FDCD7CFD71200F00E936E81
:100B200081CFD3F10101D315D26F0F0ED015D06F45
:100B3000D051D211D06F81CFD3F1F00ED315D26F37
:100B4000F00ED25D01E0F7D7936A06D8D6C1D5F191
:100B50000101010ED46F12000101D76B100ED75D99
:100B600014E2D751EA6A000FE96E010EEA22EF5053
:100B7000D05D08E1D751EA6A100FE96E010EEA2252
:100B8000EFCFD6F1D729D76FE9D7D6C181FF640E51
:100B9000E66EE66A51DEE552E55212000101D86BBD
:100BA000070ED85D1DE288DF0101D96FD851EA6ACE
:100BB000DA0FE96E010EEA22D9C1EFFFD851EA6AD5
:100BC000DA0FE96E010EEA22EF50460802E108D082
:100BD00004D0D9C1E6FF40DFE5520101D82BE0D7B0
:100BE000D851EA6ADA0FE96E010EEA22EF6A1200C2
:100BF0000101D86B070ED85D16E2D851EA6ADA0F08
:100C0000E96E010EEA22EF50E66E26DFE5520101A1
:100C1000D829EA6ADA0FE96E010EEA22EF5001E103
:100C200002D0D82BE7D71200D9CFE6FFE1CFD9FF0A
:100C3000E652F250800B01E0010EDF6EF29EA69E9E
:100C4000A69CA684FE0EDB50A96EFD0EDB50A86E9E
:100C5000550EA76EAA0EA76EA682A6B2FED7A694C0
:100C6000DF50E8B0F28EE8A0F29EE552E552E7CF01
:100C7000D9FF1200D9CFE6FFE1CFD9FFA69CA69EEF
:100C8000FE0EDB50A96EA680A85000D0E552E7CF3B
:100C9000D9FF12004D0EE66EE66A6C0EE66E65EC4C
:100CA00008F0E552E552E5521200D9CFE6FFE1CF58
:100CB000D9FF040EE126DE6ADE6ADE6ADD6ADD52F5
:100CC000DD52D9CFE9FFDACFEAFFD890030EEB501F
:100CD000000A08E6400EEE5C0D0EEE58030EEE58CC
:100CE000000EEE5811E29EAA04D0D9EC08F00ED006
:100CF00001D000D0D9CFE9FFDACFEAFFEE2A000E0B
:100D0000EE22EE22EE22DDD7000E00D0006E040EA1
:100D1000E15C02E2E16AE552E16E0050E552E7CFA4
:100D2000D9FF1200D9CFE6FFE1CFD9FFE6529EAA44
:100D3000FED7D9EC08F0DF6EDFCFE6FFF8EC08F065
:100D4000E552F5D7DF5000D0E552E552E7CFD9FFA5
:100D50001200D9CFE6FFE1CFD9FFE6529EAAFED717
:100D6000D9EC08F0DF6EDF5000D0E552E552E7CF56
:100D7000D9FF1200A6DD0DDE0101F76BF86B080E3E
:100D8000F8AF02D0D89003D0F75D000EF85917E203
:100D9000F7C1E9FFF8C1EAFFD890E936EA36C00E9C
:100DA000E926010EEA22EECFE6FFEFCFE6FF8BD871
:100DB000E552E5520101F72B000EF823E0D70EDED5
:100DC000200EE66E010EE66E59DEE552E55262DF58
:100DD0000D0EE66EE30EE66E010EE66EAAEC08F06E
:100DE000E552E552E552D5DDF9DD3E0EE66E34DE24
:100DF000E552010E0101F96FFA6B080EFAAF02D04D
:100E0000D89003D0F95D000EFA590FE2E30EF925F0
:100E1000E96E010EFA21EA6EEF50E66E1DDEE55234
:100E20000101F92B000EFA23E8D7E66A010EE66EFF
:100E3000DFDDE552E552080E0101F96FFA6B0D0E88
:100E4000FAAF02D0D89003D0F95D000EFA590FE244
:100E5000E30EF925E96E010EFA21EA6EEF50E66E17
:100E6000FBDDE5520101F92B000EFA23E8D7D00E85
:100E7000E66E070EE66EE0DCE552E5520101F76B27
:100E8000F86B080EF8AF02D0D89003D0F75D000ED3
:100E9000F85917E2F7C1E9FFF8C1EAFFD890E9363F
:100EA000EA36C00EE926010EEA22EECFE6FFEFCFCA
:100EB000E6FF73D8E552E5520101F72B000EF82347
:100EC000E0D77DD71200D9CFE6FFE1CFD9FF020EE0
:100ED000E12684DD2A0EE66EBFDDE552040EDE6EED
:100EE000DD6ADECF00F0DDCF01F0D890015004E6DE
:100EF0000C0E005C000E015815E2FD0EDBCF00F079
:100F0000FE0EDBCF01F0DE500024E96EDD50012043
:100F1000EA6EEF50E66EA0DDE552DF2A010E01E336
:100F2000DB2ADFD7E66A010EE66E62DDE552E552A6
:100F30000B0EDE6EDD6ADECF00F0DDCF01F0D89063
:100F4000015004E6120E005C000E015815E2FD0E81
:100F5000DBCF00F0FE0EDBCF01F0DE500024E96EA7
:100F6000DD500120EA6EEF50E66E76DDE552DF2AB5
:100F7000010E01E3DB2ADFD7E80EE66E030EE66E14
:100F80005BDCE552E552020EE15C02E2E16AE55209
:100F9000E16EE552E7CFD9FF1200D9CFE6FFE1CFEE
:100FA000D9FF020EE76EFD0EDBCFE9FFFE0EDBCFB1
:100FB000EAFFE750E926000EEA22EF500101EE5D5C
:100FC00002E0000E01D0010E006E030EE76EFD0E72
:100FD000DBCFE9FFFE0EDBCFEAFFE750E926000E8C
:100FE000EA22EF50EF5D02E0000E01D0010E001486
:100FF00019E0F7C1E9FFF8C1EAFFD890E936EA360F
:10100000C00EE926010EEA22EECFE6FFEFCFE6FFA3
:101010005ADFE552E552E80EE66E030EE66E0CDC92
:0C102000E552E552E552E7CFD9FF12007F
:04102C002A0EF66E24
:10103000080EF76E000EF86E02010900F550056FFC
:101040000900F550066F03E1056701D03DD00900A6
:10105000F550006F0900F550016F0900F550026F5F
:1010600009000900F550E96E0900F550EA6E090023
:1010700009000900F550036F0900F550046F0900DD
:101080000900F6CF07F2F7CF08F2F8CF09F200C255
:10109000F6FF01C2F7FF02C2F8FF0201035302E1AB
:1010A000045307E00900F550EE6E0307F8E2040769
:1010B000F9D707C2F6FF08C2F7FF09C2F8FF02011D
:0A10C0000507000E065BBFD7120003
:0610CA00D9CFE6FFDACFEA
:1010D000E6FFE1CFD9FFE2CFDAFFAC6AAB6AFD0EE3
:1010E000DBB0AC88DBA202D0AC8CAB8CDBB4AC8EBA
:1010F000DBA602D0AB8801D0AB8ADBB8AC849E986B
:10110000DBBAAB86DBAC02D09D8A01D09D9A9E9A59
:10111000DBAE02D09D8801D09D98FB0EDB50AF6EF8
:10112000FB0EFC0EDBCF01F001C000F0016A0050A5
:10113000B06EAC8AAB8E949C948EAC50100B04E0D5
:10114000AC50800B01E1948CE552E5CFDAFFE7CF9C
:04115000D9FF1200B1
:0C115400D9CFE6FFDACFE6FFE1CFD9FFEC
:10116000E2CFDAFFE652E652DF6AFB0EDB50DF5CCD
:1011700018E29EAAFED7D9EC08F0E76E010EE7CF81
:10118000DBFFFC0EDBCFE9FFFD0EDBCFEAFF010E3C
:10119000DBCFEFFFFC0EDB2AFD0E01E3DB2ADF2AAB
:1011A000E4D7E552E552E552E5CFDAFFE7CFD9FFC4
:0211B00012002B
:0E11B200D9CFE6FFDACFE6FFE1CFD9FFE2CFDB
:1011C000DAFFE652F20E0101FB17ABAC03D0FB9144
:1011D000ABB0FB81ABB4FB85ABB2FB87AE50DF6E2F
:1011E000DF50E552E552E5CFDAFFE7CFD9FF120035
:1011F000D9CFE6FFDACFE6FFE1CFD9FFE2CFDAFFC2
:10120000ACAC04D0AC900101FBB3AC80FD0EDB5064
:0E121000AD6EE552E5CFDAFFE7CFD9FF120051
:02121E00FF0EC1
:10122000E350066E480E01D04C0EE76EE72EFED757
:0E123000E76AE72EFED7062EF7D70000120061
:02123E00000EA0
:10124000F36E00EE00F0080E01D81200EA6002D042
:0E125000EE6AFCD7F350E9601200EE6AFCD79C
:02125E0012EE8E
:1012600040F022EE40F0F86A059C16EC08F048ECDD
:0A12700009F0BAEC06F0FBD71200FB
:06127A00FF0EE350E84EF8
:101280001200000000D000D000D0E82EFAD71200E3
:0212900012004A
:0E129200EEEDEBE7DEDDDBD7BEBDBBB77E7D4C
:1012A0007B77303132333435363738394142434435
:1012B00045463E3E5441473C3C00313941454A4F4A
:1012C0005345204845524E414E44455A004631460A
:1012D000395041424C4F204A494D454E455A200015
:1012E0003142414350414F4C4120455350494E4FAC
:1012F0005A4100314141444A41494D4520424554FB
:10130000414E5A4F5300464646464C55495320528B
:101310004F424C45444F20200046464646524F42DD
:101320004552544F204C494D4F4E200046464646AC
:101330004A4F484E2043415354454C4152200046A9
:10134000464646444149535920504552455A20206B
:10135000200028013B014E016101740187019A01BF
:02136000AD01DD
:00000001FF
